:100000000200F93200000000000000320000000091
:10001000000000320000000000000032000000007C
:10002000000000320000000000000032000000006C
:1000300000000000000000000000000000000000C0
:10004000000000320000000000000032000000004C
:10005000000000000000000000000032000000006E
:10006000000000320000780F790BE766A2E7500627
:10007000E7A2E774FF22E50BB50F12E50AB50E0DF6
:10008000E509B50D08E508B50C03C3E42274FF22A9
:1000900012006660044002E422740122AE02E6F718
:1000A0000809DEFA22740D1200B0740A1200B022A0
:1000B0003099FDC299F599227B0474FA11CCDBFAD0
:1000C000DAF622C0E0740311CCD0E02278817916F0
:1000D000D8FED9FCD5E0F522E6F760040809DAF885
:1000E000E4F7227900E6080970FBE91422E624010E
:1000F000F6FA08E63400F64A2278FFE4F6D8FD75F1
:10010000813DC28E759852758922758D00D28E758B
:100110002000758BFC758DFCC281C2803161780B2B
:10012000E88360061200B00880F602013353746160
:1001300072740011A5D283D284D2857A0111B8C21B
:1001400083C284C2857A0111B8780BE883600612F5
:1001500000B00880F602015A5800020135C2AF8093
:10016000FE740F11CC7521305132740A11CC7521F7
:10017000305132740111CC7521305132740411CCDC
:100180007521205132740111CC7521205132752115
:10019000805132740111CC7521005132752180518A
:1001A00032740111CC75210051327521C051327465
:1001B0000111CC7521005132752110513274011199
:1001C000CC79247B05EB04FB83F70970F880115789
:1001D0003731303020616E6420426173636F6D008F
:1001E000753901753A00853908853A09E53A7F0085
:1001F00030E7027FFF8F0A8F0B782411E3F50C752F
:100200000D00750E00750F00119070030202317A17
:10021000017424C0E08539F0D0E025F014F8793B72
:100220001200D8783BE6F522513E783911ED0201F3
:10023000E6228521A0D282740111CCC282228522BD
:10024000A0D282D280740111CCC282C2807401110A
:10025000CC7F047822E623DFFDF68522A0D282D26D
:1002600080740111CCC282C280740111CC220000C2
:00000001FF
